:1000000000308A008E2900000A108A100A11820727
:1000100050344B34493454342D3435345234203434
:100020000D340034263084000008031926280130DE
:10003000F800F701F70B1A28F80B19284A30F700D7
:10004000F70B202800000000800B172800348316CF
:100050000513831205130830F800000000000000AB
:10006000F8174128F813AB0C03180517031C0513E8
:10007000781741287813F80B33280000000000009F
:1000800005171C308400840B43280000F81B32281D
:10009000781B3A280034603083168F000F0804392B
:1000A000043C031D4E2802308312A500FA30A6003E
:1000B0001220A50B56280230A500A50803197028A8
:1000C0008316851083128510FA30A600122083163D
:1000D000851083128514FA30A6001220A5035D282E
:1000E000A50125080420A50AF700AB002720083049
:1000F0002502031D71280330A6002E30AB002720F7
:10010000A60B7D280D30AB0027209829AD01AC014E
:10011000831605140030831205180130013C031DBD
:100120009528AC0A0319AD0A8828831605140030F7
:10013000831205180130003A031DA228AC0A0319E6
:10014000AD0A95282C08F8002D08F9000034A90103
:10015000AA012A08073C031CBE280310A90C86200C
:100160007908AC007808AB00AC08031DBB282B084D
:10017000353C0318BC28A917AA0AA9282908F800A1
:100180000034AA1BD3280F30F700290EF7050A30D8
:1001900077020318CE283030F707D0282A08F7074F
:1001A0007708AB0027200F30A9050A302902031871
:1001B000DB283030DD28AA132A08A9072908AB005C
:1001C00027200034AB012B08043C031CFE288620AA
:1001D0007908AA007808A900AA08031DF3282908AD
:1001E000203C0318FC28AA08031DFC282908253CEC
:1001F000031CFC28AB0AFD28AB01E328AA08031D59
:100200000B292908343C031C0B2986207908AA00F5
:100210007808A900FE288316851083128510A72070
:100220007808A500A7207808A600A7207808A700CE
:10023000A7207808A8002508533C031D7329260829
:10024000353C031D7329FF30831686008312060890
:100250002702031D73293A30AB0027203130AB0051
:1002600027202708A9003730AA00C1202808A900A4
:100270003730AA00C1200D30AB0027200A30A9007A
:100280001730AB007030AA00AA08031D4A29AB083A
:1002900003196B2983168513831285130130AC0073
:1002A0002C082902031C5A292A080319AB03AA03A4
:1002B000AC0A502983168513831285170130AC00D0
:1002C0002C082902031C6A292A080319AB03AA0374
:1002D000AC0A6029442983168510831285142808E6
:1002E000F8008D298D293A30AB0027203030AB0043
:1002F00027202708A9003730AA00C1202808A90014
:100300003730AA00C1200D30AB002720831685109E
:1003100083128514FF30F8008D299D2984011F3038
:100320008305073083169F000513831205174B289A
:100330000130A200A300A400E2287808A100210B4C
:10034000CD298316851600308312851A0130013CB1
:10035000031DBC2983160511831205110230A50067
:10036000FA30A6001220A50BB029831605118312BE
:1003700005150130A200CC29A208031DC2290130B5
:10038000A200C329A201A208031DC8290511C92979
:1003900005158316051183126B2A2108023C031DE3
:1003A000FD298316851600308312851A0130013C21
:1003B000031DEC2983168511831285110230A500D7
:1003C000FA30A6001220A50BE029831685118312AE
:1003D00085150130A300FC29A308031DF229013073
:1003E000A300F329A301A308031DF8298511F92906
:1003F00085158316851183126B2A2108033C031D82
:100400002D2A8316851600308312851A0130013C8F
:10041000031D1C2A83160512831205120230A50043
:10042000FA30A6001220A50B102A8316051283129B
:1004300005160130A4002C2AA408031D222A01302D
:10044000A400232AA401A408031D282A0512292A8E
:1004500005168316051283126B2A2108043C031D1E
:10046000372A8316051183120511A2016B2A210870
:10047000053C031D412A8316851183128511A301B2
:100480006B2A2108063C031D4B2A83160512831292
:100490000512A4016B2A2108073C031D562A831666
:1004A0000511831205150130A2006B2A2108083CB2
:1004B000031D612A83168511831285150130A3005F
:1004C0006B2A2108093C031D6B2A8316051283122F
:0A04D00005160130A4009C2963000A
:02400E00103967
:00000001FF
